:100000000C9408030C9484080C943A030C943A035F
:100010000C94EE070C943A030C943A030C943A03B4
:100020000C943A030C943A030C943A030C943A035C
:100030000C943A030C943A030C943A030C943A034C
:100040000C94642B0C943A030C94FE2D0C94302EDB
:100050000C943A030C943A030C943A030C943A032C
:100060000C943A030C943A0305A84CCDB2D44EB983
:100070003836A9020C50B9918688083CA6AAAA2A4B
:10008000BE000000803F98039C03700319030F0318
:10009000BF0271023102E5018F01470139012C01D4
:1000A0002601200117011201060189017B016D0162
:1000B00065015B014E01DD01D301C401BB01B0014B
:1000C000A801A1019801240218020502F901ED011D
:1000D00064025B027B0339024E024102AC029F02C2
:1000E0008E027C029F0276027B030703FF02EF026F
:1000F000E602E202D502C70267035A034D0340033A
:1001000036032D0324035445585420414C41524D8D
:100110005300414D5053004D41482058313030007C
:1001200054494D455200535045454400414C5449B3
:1001300054554445205831300044495354414E43AE
:1001400045205831303000414C41524D5300544805
:10015000524F54544C452050574D004F5344205457
:1001600058204348004D41472043414C00444542FC
:10017000554700312E31560035560056205245461F
:1001800000494D50004D455400554E4954530041CF
:100190004456414E434544004D4150204D4F444547
:1001A0000047494D42414C0053454E534F52530076
:1001B00047505320434F4F524453005448524F54DA
:1001C000544C45005343524F4C4C494E47204241FA
:1001D00052530053494445204241525300484F5224
:1001E000495A4F4E00444953504C41590041444AEA
:1001F000555354205A45524F0041444A55535420B8
:10020000414D505300555345205649525455414C89
:100210002053454E534F5200444953504C415920AE
:100220004D414800444953504C415920414D505391
:100230000043555252454E54005553452050574D9A
:10024000005345542052535349204D494E005345C5
:10025000542052535349204D415800534554205285
:1002600053534900444953504C4159205253534928
:1002700000525353490043454C4C5300444953509A
:100280004C41592056494420564F4C5453004D413F
:10029000494E20564F4C545320414C41524D004141
:1002A000444A55535420564F4C54530044495350DC
:1002B0004C4159204D41494E20564F4C5453005605
:1002C0004F4C54414745005448524F54544C4520DC
:1002D0004558504F005448524F54544C45204D49B6
:1002E0004400545041005941572052415445005256
:1002F0004F4C4C20504954434820524154450052E1
:1003000043204558504F005243205241544500521B
:10031000432054554E494E470050494420434F4EC8
:10032000464947004D415820414D5053004D4148EA
:100330002055534544004D415820535045454400F5
:100340004D415820414C544954554445004D415865
:100350002044495354414E434500544F542044498E
:100360005354414E434500464C592054494D450095
:10037000535441544953544943530055534520461F
:1003800043003C504147453E00534156452B45589C
:1003900049540045584954004F4646004F4E00D33B
:1003A00003CA03B803A7034E4F54204445544543A2
:1003B0005445442D50414C004E4F54204445544523
:1003C000435445442D4E545343004155544F2D50F2
:1003D000414C004155544F2D4E545343002604EDDB
:1003E0000315040604F603ED03F203EE030053497C
:1003F0003A0049443A00202020202B5049544348D9
:100400002046554C4C00202020202B59415720528B
:1004100049474854004D454E553A54485254204D92
:100420004944444C45004D572D4F5344202D2052F4
:10043000312E362E3800A30481047A049B049304E1
:100440008A0454044E04A304710467045E04444502
:10045000425547004C4F5720564F4C545300204DA7
:10046000495353494F4E004155544F20484F4C4437
:10047000004155544F20525448002041524D4544AC
:100480000044495341524D4544004C4F572053417D
:10049000545300204E4F20475053004E4F204441AC
:1004A000544100001D1A1D1C1D191D1C1D1B1D1C67
:1004B0001D181D1C1D1A1D1C1D191D1C1D1B1D207A
:1004C000007BC12A00210090005400240072002704
:1004D000003500CB0060017EC17EC137C110011D17
:1004E0000102000F004C01F2006BC12FC175017FAA
:1004F00001C200BB00BB00030007007A00550106E3
:10050000015C003400C50064005701BA001801DC2A
:10051000C020C034C036C0B7C090C054C024C07220
:10052000C028C0CBC0CAC060C17EC17EC137C11067
:10053000011D0102C00FC04DC1F3C06BC12FC171BD
:10054000C178C1C2C0BBC0BBC0030007007AC055A0
:10055000C106C15CC03400C30064C05301BA0018B6
:10056000C1DCC000000000960000000004F4015847
:10057000020C00003C000000018A04C800000000DA
:10058000000100C800326401010100000001000008
:100590000001010000010000010000000000010155
:1005A000010101000101000400000005000100003C
:1005B00000001E4D574F5344002020202000000013
:1005C0000800020100000304070000000000000012
:1005D00000010204081020408001020408102001DC
:1005E00002040810200404040404040404020202A7
:1005F0000202020303030303030000000025002896
:10060000002B0000000000240027002A0000602EBC
:10061000E7E5F7E085EA98E001C08193EF3FF9074D
:10062000E0F3D9F311241FBECFEFD8E0DEBFCDBF7A
:1006300011E0A0E0B1E0EAEBF5E602C005900D9212
:10064000AA35B107D9F727E0AAE5B1E001C01D92AC
:10065000A735B207E1F713E0C8E0D3E004C0219763
:10066000FE010E945B32C730D107C9F70E94CF2E2E
:100670000C94DB320C9400000C94CD326091A304F6
:100680007091A4046115710581F420E030E044EB21
:1006900053E460916A0470916B0480916C049091B2
:1006A0006D040E947D2F0E94EF2F2091DC0584E6CF
:1006B000289F9001112481E0261737070CF080E075
:1006C00008958091C70481110EC080918106811127
:1006D0000AC080918006811106C080E88093470699
:1006E00081E080938006089580918006882309F434
:1006F00042C080E090E1A0E0B0E080931A029093C5
:100700001B02A0931C02B0931D028091D30581119E
:1007100004C08091CD05882389F080911A029091C0
:100720001B02A0911C02B0911D02916080931A02DD
:1007300090931B02A0931C02B0931D02809116029D
:1007400090911702A0911802B091190240911A02DB
:1007500050911B0260911C0270911D02842395230D
:10076000A623B7238093160290931702A093180232
:10077000B0931902089580918106882329F08FE9AA
:1007800096E0A6E2B0E0B9CF8AE090E0A2E0B0E067
:1007900080931A0290931B02A0931C02B0931D0237
:1007A0002091D00421FF0CC08AE190E0A2E0B0E0EB
:1007B00080931A0290931B02A0931C02B0931D0217
:1007C00080919106813089F080911A0290911B02EC
:1007D000A0911C02B0911D02816080931A02909337
:1007E0001B02A0931C02B0931D0223FF11C0809135
:1007F0001A0290911B02A0911C02B0911D02806A06
:1008000080931A0290931B02A0931C02B0931D02C6
:1008100080911406811179CF80911A0290911B0268
:10082000A0911C02B0911D02986067CF8091BF0417
:10083000882369F18091C704882349F16091AD0450
:100840007091AE046115710511F12091E50580E00C
:1008500090E0222379F10E94253021EB32E047E538
:100860005BE30E9416319B01AC0160910A0270911A
:100870000B0280910C0290910D020E94072F609351
:100880000A0270930B0280930C0290930D02609108
:100890000A0270910B0280910C0290910D020E944D
:1008A000F62F6093500470935104809352049093F8
:1008B000530408950E9425302FE632E143E85AE3BD
:1008C000D0CFEF92FF920F931F93CF93DF9308EC5B
:1008D00015E0C0E0D0E0CE012196CD34D10531F055
:1008E000F80161918F010E943C03F5CF0AEB15E0FE
:1008F000CCE4D0E0F8016081CE010E943C03F80115
:1009000061810E5F1F4FCE0101960E943C0322962B
:10091000CA35D10579F76CE080E090E0DF91CF91A6
:100920001F910F91FF90EF900C943C03CF92DF92B8
:10093000EF92FF920F931F93CF93DF93C0918306A3
:1009400082E5C89FE001112438E6E32E35E0F32E5E
:100950008E0104551F4FC65ADF4FC017D10759F1FA
:10096000CE010E94C532C82ED12CF701D182C0829F
:10097000CE0101960E94C53290E0982F88278C0DF9
:100980009D1DF701918380832091E605222359F074
:100990009C0131702739310530F0213F310540F499
:1009A0004E9691838083F2E0EF0EF11C2296D5CF14
:1009B000CC96F701F6CFDF91CF911F910F91FF9069
:1009C000EF90DF90CF900895EF92FF920F931F93D7
:1009D000CF93DF9308EC15E0C0E0D0E0CE010E9499
:1009E000C532F80181938F012196CC34D105B1F73E
:1009F0000AEB15E0CDE4D0E0CE0101970E94C532AC
:100A0000E82EF12CF801F182E082CE010E94C5327D
:100A100090E0982F88278E0D9F1DF8018193919368
:100A20008F012296CB35D10539F7DF91CF911F91F8
:100A30000F91FF90EF900C949604CF92DF92EF927B
:100A4000FF920F931F93CF93DF9380E090E00E947B
:100A5000C5328C3009F458C0C0E0D0E0CC34D105A8
:100A600049F0FE01EF58FA4F6491CE010E943C0319
:100A70002196F4CFFE01E95EFA4F05911491602FA3
:100A8000CE010E943C03612FCE0101960E943C03DF
:100A90002296CA35D10571F78E010A551109C80190
:100AA0008F5E9A4F7C01FC01C590D4906C2DCE01D5
:100AB0000E943C036D2DCE0101960E943C03F8017B
:100AC000E154FB4F05911491602FCE018E5A9F4F38
:100AD0000E943C03612FCE018D5A9F4F0E943C0320
:100AE000F70105911491602FCE018C559F4F0E9404
:100AF0003C03612FCE018B559F4F0E943C032296F1
:100B0000CE3FD10509F0C8CFDF91CF911F910F9152
:100B1000FF90EF90DF90CF9008954F925F926F9289
:100B20007F92AF92BF92CF92DF92EF92FF920F939C
:100B30001F93CF93DF93C2EED4E041E0E42E41E077
:100B4000F42E00E010E05AE0D52E0530110509F42E
:100B500054C0F70181917F010E94472B2091090227
:100B600001112CC03091D305332319F08091CA04B0
:100B700090E0D09EF001D19EF00D1124E20FF11D06
:100B8000EE0FFF1FEE52FB4F2881398140815181CA
:100B9000241B350B3983288320813181820F931FD9
:100BA000969587959183808328813981820F931F41
:100BB000998388830F5F1F4F6496C7CF0430C9F6AF
:100BC0003091CE05332381F08091640490916504C7
:100BD00095958795009741F4E22FF0E0EE0FFF1F07
:100BE000EE5DFA4F808191813091CD05332309F27A
:100BF0008091A1049091A204BCCF8091D305C090B4
:100C0000E204D090E304C091ED05811116C160911A
:100C1000D205E12CF12C70E080E090E0C111FAC027
:100C20000E9427302B013C01C701B6010E942530EC
:100C30009B01AC01C301B2010E94163127E137EBE1
:100C400041ED58E30E9416310E94F62F7093630421
:100C5000609362048091CA0580935E04C090F6049C
:100C6000D090F7046091DA05E12CF12C70E080E07F
:100C700090E0C111ECC00E9427302B013C01C7015C
:100C8000B6010E9425309B01AC01C301B2010E9454
:100C9000163127E137EB41ED58E30E9416310E94EF
:100CA000F62F70936104609360048091D5058111E3
:100CB00062C18091D705C091BC05D091BD0500915E
:100CC000BE051091BF058111DEC040900A0550900D
:100CD0000B0523E0559447942A95E1F7052C000C69
:100CE00066087708C301B2010E94273060936E0442
:100CF00070936F0480937004909371049E0140E0A0
:100D000050E0C8011F921F929F930F93A12CB12C0A
:100D10006501E12C14E0F12E00E010E0C301B20106
:100D20000E948D2E0E9427306B017C010F900F9046
:100D30000F900F9020E030E0A9010E94732F87FDF3
:100D400099C0C0926E04D0926F04E0927004F09249
:100D500071048091CC05882309F445C06091320567
:100D60007091330583E0759567958A95E1F77093E7
:100D700067046093660480918106882349F080911E
:100D80009B068F3009F00BC17093C3056093C205B9
:100D9000E090C205F090C30500E010E02091C0058E
:100DA0003091C10540E050E0072E000C880B990BF4
:100DB0001F921F921F92E4E6EF93A12CB12C6501C4
:100DC0000E948D2E0F900F900F900F906536710539
:100DD00014F064E670E077FF02C060E070E07093AA
:100DE000670460936604809109028F5F883008F081
:100DF000E0C080930902DF91CF911F910F91FF9086
:100E0000EF90DF90CF90BF90AF907F906F905F900A
:100E10004F9008950E9427302B013C01C701B60175
:100E20000E9425309B01AC01C301B2010E94163122
:100E30002FE632E143E05AE305CF73E0D594C7943F
:100E40007A95E1F7D0926304C092620403CF0E94C6
:100E500027302B013C01C701B6010E9425309B01C0
:100E6000AC01C301B2010E9416312FE632E143E02A
:100E70005AE313CF10926E0410926F041092700414
:100E80001092710466CF80911601909117016091C4
:100E90000801709109018617970740F060910601DB
:100EA000709107018617970708F4BC0180E090E075
:100EB000685E734081099109623FF3E07F07810515
:100EC000910508F04DC02AE030E040E050E00E947B
:100ED0001A3269017A01A7019601C701B6010E9481
:100EE000D4310E9425302AE037ED43EA5CE30E94CA
:100EF00016312B013C01C701B6010E9425309B0130
:100F0000AC01C301B2010E94072F6B017C01B80143
:100F100080E090E00E9425309B01AC01C701B60142
:100F20000E9416312AE037ED43E25CE30E9416315D
:100F30006B017C018091C704BE018823B9F080E079
:100F400090E00E942530A70196010E94072F609330
:100F50006E0470936F048093700490937104F9CEC3
:100F600094E6C92ED12CE12CF12CB5CF80E090E095
:100F70000E942530ECCF809168049091690497FF1E
:100F80000CC005976AE070E00E940632072E000C44
:100F9000880B990B0E942730DACF0596F3CF81306A
:100FA00009F0F6CE7093C1056093C00510929B06C0
:100FB000EFCE109209021FCF3B98F89480916C00FD
:100FC00083FD0AC0809168008260809368008091F0
:100FD0006C00886080936C00789408951F920F9243
:100FE0000FB60F9211242F933F934F935F936F93FC
:100FF0007F938F939F93AF93BF93CF93EF93FF9381
:10100000C6B178940E94BA2B209105023091060255
:10101000AB01421B530B9A01293B3B4018F021E0E6
:10102000209300017093060260930502C3FD3CC04B
:101030002091070230910802621B730BCB018F5E77
:101040009240209100018B3D954080F4809187066D
:10105000882329F1822F90E0893091053CF4880F94
:10106000991FFC01E25FFE4F718360832F5F209325
:1010700000017093860660938506FF91EF91CF91F2
:10108000BF91AF919F918F917F916F915F914F91A0
:101090003F912F910F900FBE0F901F901895709356
:1010A000650460936404E2CF7093080260930702C2
:1010B000E4CFCF93DF93C0E0D0E060E0CE010E94A8
:1010C0003C032196C11582E0D807B9F7DF91CF9193
:1010D00008958EBD0DB407FEFDCF8EB50895DC01D9
:1010E000FB01EE5CFD4F9D91992311F09193FBCF95
:1010F0000895DB01AE5CBD4FFC01249101962223D3
:1011000011F02D93F9CF08951F920F920FB60F9201
:101110001124109201020F900FBE0F901F9018958E
:10112000CF93C62F0E9469088C2FCF910C94690829
:101130005E9A2A9864E670E080E090E00E94DF2BDF
:101140002A9A80E58CBD81E08DBD8DB58EB56AE0B3
:1011500070E080E090E00E94DF2B5E9864E670E033
:1011600080E090E00E94DF2B80EA0E9469088FEF08
:101170000E9469088370813001F58093E6058093B1
:101180009406809302028091E605882319F180EE8F
:1011900091E090930402809303026CE480E00E944B
:1011A00090085E9A9FB7F894E89A809169008260EF
:1011B000809369009FBF0C949604823029F41092AA
:1011C000E60510929406DDCF9091E6059E5F909320
:1011D0009406D7CF86E891E09093040280930302AF
:1011E0006CE0DCCF0F931F93CF93C82F5E98609174
:1011F000E605611160E480E00E9490086C2F89E0B0
:101200000E9490080AE416E0C0E06C2F8AE00E9479
:101210009008F80161918F018BE00E949008CF5FE8
:10122000C63399F760EA88E00E94900880EA0E943D
:10123000690885FDFBCF8091E60581110EC06CE049
:1012400080E00E9490085E9A64E170E080E090E0A7
:10125000CF911F910F910C94DF2B6CE4F1CF5E982E
:1012600080EA0E9469088FEF0E946908837090915C
:10127000020289130C94980880E80E9469088FEF95
:101280000E94690883FFF6CF0895EF92FF920F93B3
:101290001F93CF93DF93FB0197FF37C09195819503
:1012A0009109C1E0DF01A40FB11D1C92DEE20AE04A
:1012B00010E0421306C04150DF01A40FB11DDC93C2
:1012C00020E03FEF340F7F01E30EF11CB8010E94D4
:1012D0000632805DD7018C93CB013323D1F02111ED
:1012E00016C00097A1F4CC2339F03EEF340FDF0194
:1012F000A30FB11D8DE28C9380E2332351F0315066
:10130000DF01A30FB11D8C93F8CFC0E0CBCF432FEB
:10131000D0CFCF01DF91CF911F910F91FF90EF9030
:1013200008958F929F92AF92BF92CF92DF92EF92E9
:10133000FF920F931F93CF93DF936A01D22F97FFF2
:1013400008C090958095709561957F4F8F4F9F4F06
:101350000E2D24E630E040E050E00E943C32CA010D
:10136000B90126E02D0FF601E20FF11D108225E0F4
:101370002D0FF601E20FF11D0083C4E0CD0F2AE02E
:10138000822E912CA12CB12C3EE2F32E2C2F30E09A
:1013900041E04C0FD41306C02C0D3D1DF901F08225
:1013A000C150F4CF8601020F131FA50194010E94C2
:1013B0003C32605DF8016083B901CA01CC2391F031
:1013C000C33070F7611571058105910549F7C1506A
:1013D000EC2FF0E03196EC0DFD1D80E28293CE16ED
:1013E000DF06E1F7C601DF91CF911F910F91FF90CA
:1013F000EF90DF90CF90BF90AF909F908F90089527
:101400002F923F924F925F926F927F928F929F9214
:10141000AF92BF92CF92DF92EF92FF920F931F9302
:10142000CF93DF9300D000D0CDB7DEB76B017C0146
:101430001A012B83222309F47BC018E0F101E10F8C
:10144000F11D10821C830B8196E0492E512C612CDA
:10145000712C2CE3822E912CA12CB12C8C818150EB
:101460009101280F311D87FD3A953A832983C701E1
:10147000B6012AE030E040E050E00E941A32605DA0
:10148000E981FA8160838C818250B101680F711DFE
:1014900087FD7A957A836983CA01B901A301920114
:1014A0000E941A32605DE981FA816083C701B6014A
:1014B000A50194010E941A3269017A01FC81F3505E
:1014C000FC83F1012C81E20FF11D27FDFA953AE32F
:1014D0003083015018F68B81880F880F6B81681B51
:1014E000160F13508AE0882E912CA12CB12C11508C
:1014F0003101610E711C17FD7A94C701B601A50177
:1015000094010E941A32605DF301608369017A01DF
:10151000C114D104E104F10469F480E2112361F003
:101520001150F101E10FF11D17FDFA958083F6CFFF
:1015300015E084CF1111DBCFC1010F900F900F90F8
:101540000F90DF91CF911F910F91FF90EF90DF905F
:10155000CF90BF90AF909F908F907F906F905F9053
:101560004F903F902F90089580E0E82FF0E0E25EEA
:10157000FD4F9081992311F08F5FF7CF0895E82FE9
:10158000F0E0EE0FFF1FE859FA4F2081318122274A
:10159000307C81E02115304C09F080E008950F93F4
:1015A0001F938091A506882309F4E3C18091190651
:1015B00090911A06A0E0B0E04091CC045091CD0487
:1015C0006091CE047091CF0484239523A623B72382
:1015D000892B8A2B8B2BD1F08091F6058823B1F0D3
:1015E0001092200286E180931E0287E180931F0201
:1015F0008EE10E94BF0A882349F06091A405709192
:10160000A50571708EE192E00E946F088091FC0543
:10161000882309F461C00091CC041091CD0420917D
:10162000CE043091CF048091150690E0A0E0B0E0A8
:1016300080239123A223B323892B8A2B8B2B71F434
:101640004091160650E060E070E040235123622391
:101650007323452B462B472B09F45DC080EA80930A
:101660001E02E1E04091170650E060E070E0402388
:10167000512362237323452B462B472B39F0AE2F82
:10168000B0E0A25EBD4F82EA8C93EF5F80911806B6
:1016900090E0A0E0B0E080239123A223B323892B24
:1016A0008A2B8B2B39F0AE2FB0E0A25EBD4F81EAC2
:1016B0008C93EF5FF0E0E25EFD4F108286E00E94C7
:1016C000BF0A882349F060917405709175057170A7
:1016D0008EE192E00E946F088091CC049091CD043D
:1016E000A091CE04B091CF0440911F0650912006E6
:1016F00060E070E0482359236A237B23452B462B67
:10170000472B59F0109220028AEA80931E028BEA3E
:1017100080931F0219C0E0E0A5CF40911B065091B5
:101720001C0660E070E0482359236A237B23452B85
:10173000462B472B09F497C08DE980931E028EE952
:1017400080931F02109220028091EF058823C9F137
:1017500081E20E94BF0A8823A1F16091AA057091DD
:10176000AB0571708EE192E00E946F0880912106B6
:1017700090912206A0912306B09124064091CC04BA
:101780005091CD046091CE047091CF0484239523B1
:10179000A623B723892B8A2B8B2B99F08AEE809373
:1017A0001E028BEE80931F02109220026091AA0508
:1017B0007091AB0571706E5F7F4F8EE192E00E9479
:1017C0006F08809197068111D4C084E20E94BF0AFD
:1017D000882309F4CEC08091CC049091CD04A091CF
:1017E000CE04B091CF0440911B0650911C0660E0DE
:1017F00070E0482359236A237B23452B462B472B34
:1018000009F0B3C040911D0650911E0660E070E0E3
:10181000482359236A237B23452B462B472B09F06A
:10182000A6C0409131065091320660913306709106
:10183000340684239523A623B723892B8A2B8B2B4D
:1018400009F497C0E3E0F0E0EE0FFF1FEA5BFB4F07
:10185000859194916091B0057091B10571701F915F
:101860000F910C94790840911D0650911E0660E07E
:1018700070E0482359236A237B23452B462B472BB3
:1018800039F0109220028DEC80931E028EEC40CF36
:1018900040913106509132066091330670913406C2
:1018A000482359236A237B23452B462B472B79F06A
:1018B0008091A5044AE060E272E090E00E949032DC
:1018C0001092220285EB80931E0286EB21CF40917D
:1018D000170650E060E070E0482359236A237B2319
:1018E000452B462B472B69F64091150650E060E0EA
:1018F00070E0482359236A237B23452B462B472B33
:1019000039F0109220028CEA80931E028DEA00CFFB
:101910004091160650E060E070E0482359236A23A6
:101920007B2310922002452B462B472B29F084EC79
:1019300080931E0285ECECCE2EEA20931E022FEA45
:1019400020931F024091250650912606609127069C
:101950007091280684239523A623B723892B8A2BED
:101960008B2B09F4F1CE89E8D3CEE1E06CCFE2E035
:101970006ACF1F910F910895BC01AAE0B6E0EEE195
:10198000F2E090E08D9181939F5F9A30D9F71092A9
:1019900028028EE192E00C946F088F929F92AF9292
:1019A000BF92CF92DF92EF92FF920F931F93CF934C
:1019B000DF937C01EB0180E580931E02CB016A304E
:1019C00071053CF06AE070E00E940632CB0161E0F4
:1019D0000BC066EF7FEF0E940632CB01D7FFF7CF37
:1019E0002DE220931F0262E070E0625E7D4F4AE0CC
:1019F0000E9490328FE00E94BF0A882349F06091D4
:101A000086057091870571708EE192E00E946F08E3
:101A100082E580931E02C7015AE0E516F1043CF00E
:101A20006AE070E00E940632CB0161E00BC066EF15
:101A30007FEF0E940632CB01F7FEF7CF2DE2209315
:101A40001F0262E070E0625E7D4F4AE00E949032C9
:101A500080E10E94BF0A882349F060918805709157
:101A6000890571708EE192E00E946F088091F50502
:101A7000811105C08091FD05882309F479C080910A
:101A8000C704811104C01092AE041092AD042091DD
:101A9000A9043091AA048091AD049091AE04A901EB
:101AA000415F5F4F4817590708F0ECC00E94AE2B0A
:101AB00060937C0470937D0480937E0490937F04F4
:101AC00082E0809381048091AD049091AE04909364
:101AD000AA048093A90480910B018150803108F4FD
:101AE000CFC080930B0140913A0550913B05609126
:101AF0003C0570913D0580913E0590913F05A09178
:101B00004005B09141058A019B010C5E1F4F2F4F8C
:101B10003F4F081719072A073B070CF0D7C00E9450
:101B2000AE2B609378047093790480937A04909339
:101B30007B0482E08093800480913E0590913F0574
:101B4000A0914005B091410580933A0590933B05E3
:101B5000A0933C05B0933D0580910A0181508031EE
:101B600008F4B2C080930A018091F505811105C087
:101B700083E180930B0180930A0100919A051091F3
:101B80009B051170D090E80589E10E94BF0A8D2164
:101B900009F4DAC0C8336FEFD60714F4C8E3DFEFF7
:101BA000C93CD10514F0C8ECD0E09E01265F3F4F40
:101BB00037FF02C0295F3F4F63E0359527956A954F
:101BC000E1F7319521953109B090FA0540E0C4E084
:101BD000D0E079E0C72ED12CEEE1AE2E842F90E03C
:101BE00009970CF0A1C0443009F445E09E2D8F2DDB
:101BF00070E7E7167EEFF70614F490E78EEFE42F18
:101C0000F0E0DE01AE1BBF0B692F782F613981E058
:101C1000780714F060E971E0A69FC001A79F900DBE
:101C2000B69F900D112497FDCF9656E09595879518
:101C30005A95E1F7820F931F899682359105F0F44A
:101C4000B6010E940632A69ED001A79EB00D1124B7
:101C5000E00FF11FEA0FFB1F8058EE5CFD4FDF0124
:101C6000AC57B1098C93BB2049F09EEF940F95308F
:101C700028F4AA55B1098C93B29780834F5FAECFF9
:101C800085E12FCF0F968217930708F02CCF0E9483
:101C9000AE2B60937C0470937D0480937E049093BC
:101CA0007F0481E0809381048091AD049091AE0423
:101CB0009093AA048093A90480910B018F5F8631D1
:101CC00008F40FCF80E10DCF85E14CCF4496A11DE4
:101CD000B11D84179507A607B7070CF045CF0E94E2
:101CE000AE2B609378047093790480937A04909378
:101CF0007B0481E08093800480913E0590913F05B4
:101D0000A0914005B091410580933A0590933B0521
:101D1000A0933C05B0933D0580910A018F5F863109
:101D200008F420CF80E11ECF82E20E94BF0A811119
:101D30000BC0F801EE5CFD4FDF01119786E28C933A
:101D40008CEB81838EE780838091E905882329F0DD
:101D50008AE10E94BF0A811117C0DF91CF911F91C4
:101D60000F91FF90EF90DF90CF90BF90AF909F903A
:101D70008F900895A80EB91E8FECF5016CC0C80DA8
:101D8000D91D8FEC8883E9CFC090A2055C2D5F70D0
:101D9000C52EC091A005CF702C2F219540910B012D
:101DA00030910A010C2C000CDD08C8018C199D092A
:101DB000DEE1BC016E5C7D4F5B017601E00EF11E41
:101DC0002D02C0011124F501E80FF91F40838E5C3C
:101DD0009D4FFC01EE0DFF1D30832F5FC21784F76E
:101DE00083E0F5018183B7016E5C7D4F4B01FB0100
:101DF000319782E080838091FD05882309F4ADCF7F
:101E00008BE10E94BF0A882309F4A7CF0E94AE2B62
:101E1000AB01BC0180917C0490917D04A0917E0473
:101E2000B0917F0488519C4FAF4FBF4F481759075F
:101E30006A077B0788F420918104CD02C001112438
:101E4000223009F097CFF801E81BF90BEC19FD09D6
:101E5000EE5CFD4F89EC80830E94AE2BAB01BC0190
:101E60008091780490917904A0917A04B0917B04D8
:101E700088519C4FAF4FBF4F481759076A077B07E0
:101E800008F06BCF80918004FEE1CF02E0011124C5
:101E9000823009F074CFF701EC1BFD0BEE5CFD4FB7
:101EA00089EC80835ACFAF92BF92CF92DF92EF92AC
:101EB000FF920F931F938091D00580935F04E09071
:101EC000D105E09288068091EA05882309F46EC066
:101ED00020910D01E29E9001112480910C01E89E59
:101EE000700111248091620490916304821793071A
:101EF00008F45AC0B701625071098617970708F4B1
:101F0000BC0181E0E81AF10800E010E0032E000CAB
:101F1000440B550B70E080E090E01F921F921F92DF
:101F2000E7E0EF93A12CB12C65010E948D2E86E98C
:101F3000861B80931E020F900F900F900F900091C0
:101F40005F0410E0E0906204F0906304E016F10694
:101F500020F48091970681112DC085E10E94BF0A6F
:101F6000811103C00E151F0528F123E044E06FE145
:101F700072E0C7010E94450989EA8093230210920A
:101F800024026091920570919305717061507109FE
:101F90008EE192E01F910F91FF90EF90DF90CF9034
:101FA000BF90AF900C946F08622FABCF87E98093FE
:101FB0001E02C5CF1F910F91FF90EF90DF90CF9041
:101FC000BF90AF900895CF93DF93C0916004D091FC
:101FD000610480915E0490E0C817D90720F48091D5
:101FE0009706811121C086E10E94BF0A8823E1F093
:101FF0008FEB80931E0223E044E06FE172E0CE019C
:102000000E94450989EA809323021092240260917C
:102010009405709195057170615071098EE192E09F
:10202000DF91CF910C946F08DF91CF910895AF921B
:10203000BF92CF92DF92EF92FF920F931F938BE0AC
:102040000E94BF0A882309F48FC080E280931F0298
:10205000809116019091170120910601309107019E
:102060002817390720F490930701809306012091E7
:102070000801309109018217930720F49093090118
:1020800080930801209106013091070123303840E8
:1020900030F022E038E030930701209306012091D0
:1020A000080130910901263B334030F426EB33E040
:1020B00030930901209308012091C704211120C009
:1020C00080E2809320029DE290932102909322026D
:1020D0008093230288EC80931E0210922402609168
:1020E0007E0570917F0571708EE192E01F910F91D6
:1020F000FF90EF90DF90CF90BF90AF900C946F085F
:102100002091DB05222339F020E044E060E272E018
:102110000E944509DFCFE0900601F090070100E042
:1021200010E0209108013091090140E050E0BC012D
:1021300080E090E01F921F921F92E4E6EF93A12CA3
:10214000B12C65010E948D2EDC01CB0120E043E023
:1021500060E272E00E94450985E2809323020F90BD
:102160000F900F900F90B6CF1F910F91FF90EF90AF
:10217000DF90CF90BF90AF9008958091FB058823AA
:1021800009F44EC08091820590918305811592409B
:1021900008F446C08091C704882379F12091740423
:1021A00030917504C9016CE370E00E94F2318091B6
:1021B000090690E06817790720F080919706811151
:1021C0002FC020318EE03807A0F48CE980931E02E6
:1021D000B90180E090E020E04FE152E00E94000A67
:1021E000609182057091830571708EE192E00C948C
:1021F0006F0881E780931E02ECCF609176047091A6
:10220000770460312EE0720710F48BE9F3CF80E79A
:1022100080931E02CB016CE370E00E94F231D9CFB3
:102220000895CF92DF92EF92FF92C0906E04D0900B
:102230006F04E0907004F090710460915404709108
:10224000550480E090E00E942530A70196010E948D
:10225000732F87FF08C0C701B6010E94F62F709345
:1022600055046093540487E10E94BF0A8823F1F06B
:10227000C701B6010E94EF2FDC01CB0124E045E04D
:102280006EE172E00E9445098AE980932302109270
:102290002402609196057091970571708EE192E02D
:1022A000FF90EF90DF90CF900C946F08FF90EF902D
:1022B000DF90CF900895CF93DF9385E20E94BF0A0D
:1022C0008823B1F1C091B205D091B305D17060916E
:1022D00062047091630480E090E00E9425302091B8
:1022E0006E0430916F0440917004509171040E940B
:1022F000163120E030E048EC52E40E947D2F0E942D
:10230000F62FDC01CB0125E045E06FE172E00E9491
:10231000450980E280931E0287E580932302109294
:102320002402BE018EE192E0DF91CF910C946F0800
:10233000DF91CF91089588E10E94BF0A882319F1A7
:1023400084EA80931E0220E030E044EB53E4609185
:102350006A0470916B0480916C0490916D040E94EA
:102360007D2F0E94EF2FDC01CB014AE06FE172E08C
:102370000E949032609198057091990571708EE17C
:1023800092E00C946F08089583E10E94BF0A8823AD
:1023900029F18AEB80931E024AE06FE172E080919E
:1023A0006604909167040E9490320E94B40AE82F5C
:1023B000F0E0E25EFD4F95E290838F5FE82FF0E062
:1023C000E25EFD4F108260918E0570918F057170F5
:1023D000615071098EE192E00C946F08089587E0D6
:1023E0000E94BF0A882381F18091E305882361F16F
:1023F00080917204909173042091E4052223C1F02E
:1024000097FF02C088599E4F20E043E06EE172E0E2
:102410000E9445098DEB8093210210922202609167
:1024200076057091770571708EE192E00C946F08DB
:1024300020E044E06EE172E00E9445098DEB80935C
:10244000220210922302EBCF089588E00E94BF0A77
:102450008823F9F08091F9058823D9F080917204DE
:1024600090917304880F991F880F991F83509D4F77
:102470006AE570E00E9406326B557B4F80917805CB
:1024800090917905917049E050E08E5C9D4F0C94DD
:10249000873208950F931F93CF93DF930DED13E0D1
:1024A000C0E4D0E0F80185919491BE010E947908C2
:1024B0000E5F1F4F6E96C03381E0D80799F788EF03
:1024C00090E00E94BC0CE0919406F0E0EE0FFF1F3C
:1024D000E156FC4F8591949166E171E00E94790884
:1024E0008091A004882351F062E571E082E894E0D5
:1024F000DF91CF911F910F910C946F08DF91CF91D5
:102500001F910F910895CF93DF93C091A604D0E05F
:10251000C530D10524F48091970681111CC080E05C
:102520000E94BF0A8823B9F08EE180931E028FE1DA
:1025300080931F024AE060E272E0CE010E94903276
:10254000609168057091690571708EE192E0DF918C
:10255000CF910C946F08DF91CF9108951F93CF9383
:10256000DF938091BF04882309F464C08091C7047D
:10257000811104C01092AE041092AD041091E505D3
:102580006091AD047091AE0480E090E0111143C001
:102590000E9425302CEB34E743E15DE30E941631C5
:1025A0000E94F62FEB0180915C0490915D049C01E8
:1025B0002C5E3F4F2C173D07A8F530935D04209308
:1025C0005C0483E00E94BF0A8823A1F18091080681
:1025D000882341F090E08C179D0720F480919706A6
:1025E000811128C0E12FF0E0E95BFE4F80818093EC
:1025F0001E024AE06FE172E0CE010E9490326091CB
:102600006E0570916F0571708EE192E0DF91CF9150
:102610001F910C946F080E9425302DED3FE347EB8E
:102620005CE3BCCF8C179D0760F6D0935D04C0932C
:102630005C04C7CFDF91CF911F910895AF92BF92F5
:10264000CF92DF92EF92FF920F931F93CF93DF937E
:102650008AE00E94BF0A882309F447C08091F705E9
:10266000882309F442C0C0917C05D0917D05D170CA
:10267000CE5CDD4FFE017E978FE7808388838E8F4F
:102680006091C8047091C90469377105CCF5683848
:102690002FEF7207BCF1062E000C770B880B990BFD
:1026A0001F921F921F9221E12F93A12CB12C650143
:1026B00018E8E12EFF24FA940FEF1FEF28E730E02F
:1026C00040E050E00E948D2E862F66E00E94E431AB
:1026D00081502EE18202C00DD11D11248FE8891B8B
:1026E00088830F900F900F900F90DF91CF911F91E3
:1026F0000F91FF90EF90DF90CF90BF90AF90089533
:1027000068E7C9CF68E8C7CF8091BF04882309F183
:1027100084E00E94BF0A8823E1F08091E2058823CB
:10272000C1F020E043E06EE172E08091A704909157
:10273000A8040E9445098DEB809321021092220289
:10274000609170057091710571708EE192E00C944A
:102750006F0808958091BF048823F1F181E00E9401
:10276000BF0A8823C9F18091C0049091C104A0914F
:10277000C204B091C3040397A105B10520F4809170
:102780009706811129C020916A0530916B0531703F
:102790008091720490917304845E9D4F4091A704D0
:1027A0005091A804841B950B880F991F880F991FBF
:1027B0008D966AE570E00E940632CB0160E170E020
:1027C0000E940632805A80931E0210921F02B901A5
:1027D0008EE192E00C946F080895209133012A3025
:1027E00009F04BC080913201833009F440C0813040
:1027F00009F440C0823009F040C080E791E0422FE8
:1028000050E04A3051054CF5309131013130C1F57D
:10281000283019F48AE080933301809133018930A4
:1028200019F487E0809333012091330130E02E5F6B
:102830003F4F4EE1429FC001439F900D11240A96E5
:102840002091320130E02150310966E0629FA00101
:10285000639F500D1124840F951F20919806222309
:1028600029F08E5C9D4F23E0FC01208308958AE7C8
:1028700091E0C5CF8AE691E0C2CF80E090E0BFCF83
:10288000323089F483E080933201283019F48AE0F1
:102890008093330180913301893009F055C087E07E
:1028A0008093330151C0333019F430933201EDCFAE
:1028B000343071F483E080933201273019F48AE0D8
:1028C00080933301809133018930F1F586E0E8CFC0
:1028D000353069F483E080933201293011F430936C
:1028E000330180913301863079F58AE0D9CF3630D3
:1028F000E9F4293039F4809189068830A9F48AE016
:1029000080933301209133012093890683E08093E3
:10291000320130E02E5F3F4F4EE1429FC001439FA6
:10292000900D1124469699CF88E0EACF373079F49C
:1029300083E080933201293019F486E080933301DB
:1029400080913301873089F220913301E2CF383012
:1029500009F083CF83E080933201293019F487E0B6
:102960008093330180913301883071F7BECF2F926D
:102970003F924F925F926F927F928F929F92AF920F
:10298000BF92CF92DF92EF92FF920F931F93CF935C
:10299000DF93CDB7DEB72E970FB6F894DEBF0FBE2C
:1029A000CDBF8091EC05823011F1E0F4813009F463
:1029B0009AC12E960FB6F894DEBF0FBECDBFDF9141
:1029C000CF911F910F91FF90EF90DF90CF90BF902C
:1029D000AF909F908F907F906F905F904F903F90BF
:1029E0002F900895833009F478C1843011F702E004
:1029F00010E01C830B8311E08091BF048823C9F28F
:102A000082E20E94BF0A8823A1F219831D861E86D6
:102A1000A9818A2F90E0EB81FC818E179F074CF6ED
:102A20008091A7049091A804A13009F061C1209180
:102A3000C4043091C504821B930B845E9D4F68E6ED
:102A400071E00E94F2319C016AE570E00E9406325A
:102A50006130710509F471C10CF057C1672B09F49D
:102A600067C1B901330F880B990B0E9427302BEDFA
:102A70003FE049E450E40E94163120E030E044E3B6
:102A800053E40E947D2F1B012C016091C0047091C2
:102A9000C1048091C2049091C3040E9425304B016F
:102AA0005C01C201B1010E9483319B01AC01C501EF
:102AB000B4010E9416310E94F62F6B017C01C20105
:102AC000B1010E94782F9B01AC01C501B4010E94A5
:102AD00016310E94F62F8B019C011B01412C512CB9
:102AE000B60180E090E0C016D10608F037C142017F
:102AF000310124E6621671048104910408F431C1A5
:102B000034EF631631E073068104910408F42EC19A
:102B100044EC641649E074068104910408F42BC166
:102B20009301A4E2AA837901330F000B110BED820C
:102B3000FE820F8318871F921F921F9220E12F930E
:102B4000A12CB12C6501ED80FE800F81188520E05D
:102B500030E0A9010E948D2E69877A878B879C8738
:102B60001F921F921F928FE08F93ED80FE800F8146
:102B7000188520E030E0A901C201B1010E948D2E2C
:102B80000FB6F894DEBF0FBECDBF14E1611671041D
:102B90008104910408F4F4C02E85422F220F550BB6
:102BA000A985BA854A9F90014B9F300D5A9F300DE1
:102BB0001124BD854B2FBB0F550B469FF001479F3E
:102BC000F00D569FF00D1124C090AE05D090AF05CA
:102BD00001E0D022790189010F5F1F4F37FD780195
:102BE000F594E794EC0CFD1CCF0163E070E00E94CB
:102BF00006324EE1469FC001479F900D1124E80E1A
:102C0000F91E4981413009F4C0C095E0B92EC901CF
:102C100037FF04C088279927821B930B582F5178C0
:102C200057FF03C051505E6F5F5F452FCF01F7FF25
:102C300004C0882799278E1B9F0B63E00E94E43114
:102C40008D85813019F482E0891B982FAE85AF3FC6
:102C500011F441E0451B3296359718F491E0BD859B
:102C60009B1B0330110528F441E02F3F3F4F09F42F
:102C700040E0F981FF2309F48BC060ED8091EC0501
:102C8000843009F487C0142F110F410F940F192FAE
:102C9000160F0A8100931E0210921F026091AC056C
:102CA0007091AD0571708EE192E00E946F081093F3
:102CB0001E0210921F02B7018EE192E00E946F087F
:102CC000B0921E0210921F02B6018EE192E00E94A5
:102CD0006F0819811F5F19839BCE22E030E03C838F
:102CE0002B8310E089CE81E090E09C838B83F9CF29
:102CF00088599E4F2091720430917304821B930B6C
:102D000068E671E00E9406329ECE62307105F9F0ED
:102D10006330710509F0A5CE58E6E52EFF24F39443
:102D2000E21AF30A97010FEF0D871FEF1E8799CE66
:102D3000FFEFFD8701E00E8794CE84EB90E0821BCD
:102D4000930B9C0191E09D87A1E0AE878ACE245B26
:102D50003109B1E0BD87EFEFEE8783CE3B014C0137
:102D6000C8CEB1E2BA8324E630E0DDCEE2E2EA8307
:102D700024EF31E0D8CEF3E2FA8324EC39E0D3CE6D
:102D8000E0E0F0E020E030E01FCF84E0B82E3FCF5D
:102D900066ED74CF80917204909173042091C40405
:102DA0003091C504821B930B8A519D4F68E671E0F8
:102DB0000E94F2316DE270E00E94F23112E768CFBA
:102DC0009C01E62FF0E0E853FA4FE081F0E0EE0FCF
:102DD000FF1FEA57FF4F85919491B9010C94790830
:102DE000AF92BF92CF92DF92EF92FF920F931F9319
:102DF000CF93DF93CDB7DEB764970FB6F894DEBFFD
:102E00000FBECDBFE0913101EE0FFF0BE657FF4F34
:102E10008591949163E270E00E9479086BE671E01D
:102E200083E993E00E9479088091C60481110CC067
:102E300061E771E089E893E00E9479086BE771E04F
:102E400082E893E00E94790880913101811175C078
:102E500080915004909151049C838B8380915604FF
:102E6000909157049E838D8380915A0490915B04C6
:102E700098878F8380915C0490915D049A878987FD
:102E800020E030E044EB53E460916A0470916B04FD
:102E900080916C0490916D040E947D2F0E94EF2F11
:102EA0007C876B8780915404909155046AE070E0B0
:102EB0000E94F2317E876D87F8EFEF2EF0E0FF2E53
:102EC000CE0101966C010DE510E0F701859194911A
:102ED000B8010E9479084AE06EE172E0F601819142
:102EE00091916F010E949032B8016F5E7F4F0E94F6
:102EF0006F08F2E0EF0EF11C025E1F4F0F3281E00F
:102F0000180719F760914E0470914F0480E090E02B
:102F100021E04EE152E00E94000A6DE670E08EE191
:102F200092E00E946F088091A004882331F06DE444
:102F300071E082E894E00E946F0880913101813055
:102F400009F06CC0E2E1EE2EE4E0FE2E0DE510E0AB
:102F5000B801C7010E946F0898E0E90EF11C025EFB
:102F60001F4F0F32E1E01E0799F710E00EE1812FAD
:102F700090E009970CF040C0153009F417E0C12E1D
:102F8000D12CF7E0CF16D104ACF17EEFE72EE10EA5
:102F9000E09E70011124F601E25AFA4F80814AE066
:102FA0006EE172E090E00E949032B7016B597F4F62
:102FB0000E946F08F601EC5AFA4F80814AE06EE1F8
:102FC00072E090E00E949032B70165597F4F0E94F5
:102FD0006F08F601E65BFA4F80814AE06EE172E02D
:102FE00090E00E949032B7016F587F4F0E946F08A7
:102FF0001F5FBDCFE12ECCCF67E470E087E391E0A7
:103000000E946F086DE470E089E391E00E946F0810
:1030100063E570E08BE391E00E946F0880913101DD
:10302000823009F049C08091490590E09A838983F4
:103030008091480590E09C838B838091470590E0C8
:103040009E838D838091460590E098878F83809141
:10305000450590E09A8789878091440590E09C8798
:103060008B878091430590E09E878D876AEEE62EE0
:1030700060E0F62ECE0101966C010DE510E0F7013F
:1030800085919491B8010E9479084AE06EE172E05E
:10309000F601819191916F010E949032B8016C5EAE
:1030A0007F4F0E946F08F2E0EF0EF11C025E1F4F8F
:1030B0000F3281E0180719F780913101833009F050
:1030C00091C00E948D0587E980931E0223E044E0B1
:1030D0006FE172E080916204909163040E9445095F
:1030E00019EA109323021092240264E370E08EE147
:1030F00092E00E946F088FEB80931E0223E044E071
:103100006FE172E080916004909161040E94450932
:1031100010932302109224026CE270E08EE192E0A0
:103120000E946F085CEDE52E50E0F52E0DE510E0F5
:10313000F70185919491B8010E94790892E0E90E17
:10314000F11C025E1F4F0F32E1E01E0789F78091EC
:10315000D9054AE06EE172E090E00E9490326BEC9B
:1031600070E00E946F0867E081E790E00E94E0163F
:103170008091D2054AE06EE172E090E00E949032C8
:103180006FE870E00E946F088091D0054AE06EE120
:1031900072E090E00E9490326DEA70E00E946F0849
:1031A00061E18BEC90E00E94E0168091DA054AE044
:1031B0006EE172E090E00E94903269EE70E00E9451
:1031C0006F088091D1054AE06EE172E090E00E94C4
:1031D000903267E071E00E946F086BE085E291E059
:1031E0000E94E01680913101843009F06AC04AE003
:1031F0006EE172E080916604909167040E949032C3
:103200000E94B40AE82FF0E0E25EFD4F95E2908361
:103210008F5FE82FF0E0E25EFD4F108265E370E023
:103220008EE192E00E946F0840EDE42E40E0F42E23
:103230000DE510E0F70185919491B8010E9479089D
:10324000F2E0EF0EF11C025E1F4F013181E0180722
:1032500089F764E081E790E00E94E01680919B0688
:1032600090E0009709F49AC14AE06EE172E00E9492
:1032700090326FE870E00E946F0865E08DEA90E0A0
:103280000E94E01666E08BEC90E00E94E0164AE0B7
:103290006EE172E08091C2059091C3050E94903268
:1032A00069EE70E00E946F084AE06EE172E0809182
:1032B000C0059091C1050E94903267E071E00E94C4
:1032C0006F0880913101853009F05AC060916E0419
:1032D00070916F0480917004909171040E94EF2F9F
:1032E000DC01CB0123E044E06EE172E00E9445097D
:1032F0008AE9809322021092230264E370E08EE157
:1033000092E00E946F0836ECE32E30E0F32E0DE5DC
:1033100010E0F70185919491B8010E94790892E03C
:10332000E90EF11C025E1F4F033F110591F76CE09F
:1033300081E790E00E94E0166EE08FE890E00E9446
:10334000E0166FE08DEA90E00E94E0164AE06EE140
:1033500072E08091BE059091BF050E9490326BECA7
:1033600070E00E946F084AE06EE172E08091BC0557
:103370009091BD050E94903269EE70E00E946F0846
:1033800080913101863009F044C026EBE22E20E026
:10339000F22E0DE510E0F70185919491B8010E949D
:1033A0007908E2E0EE0EF11C025E1F4F0D34F1E0F1
:1033B0001F0789F760E281E790E00E94E01661E272
:1033C0008FE890E00E94E0166DE28DEA90E00E94A6
:1033D000E0166FE18BEC90E00E94E01667E189EE69
:1033E00090E00E94E01664E387E091E00E94E0161E
:1033F0006EE285E291E00E94E0168091EC054AE0E1
:103400006EE172E090E00E94903263E471E00E940D
:103410006F0880913101873009F04FC09AEAE92E98
:1034200090E0F92E0DE510E0F70185919491B80137
:103430000E94790882E0E80EF11C025E1F4F013104
:1034400091E0190789F78091E50561E770E0811146
:10345000AAC085E891E00E9479088091ED056FE8A7
:1034600070E0882309F4A2C088E791E00E947908FF
:103470006CE28DEA90E00E94E01680919C0690E05C
:10348000009709F496C04AE06EE172E00E94903223
:103490006BEC70E00E946F08809102064AE06EE1DA
:1034A00072E090E00E94903269EE70E00E946F0836
:1034B00063E187E091E00E94E0168091310188305D
:1034C00009F054C08091060690E09A838983809128
:1034D000070690E09C838B838091080690E09E8392
:1034E0008D838091090690E098878F838091DC0519
:1034F00090E09A8789878091DD0590E09C878B8793
:103500008CE9C82E80E0D82EFE0131967F010DE5B2
:1035100010E0A12CB12CF60185919491B8010E9484
:103520007908F6E0AF16B10469F04AE06EE172E0A6
:10353000F701808191810E949032B8016C5E7F4FCB
:103540000E946F08FFEFAF1ABF0A82E0C80ED11CBD
:10355000025E1F4F92E0E90EF11C0F32E1E01E0700
:10356000D1F660E185E291E00E94E01680913101A0
:10357000893014F01092310164960FB6F894DEBFD2
:103580000FBECDBFDF91CF911F910F91FF90EF90B4
:10359000DF90CF90BF90AF900C94ED136FE870E088
:1035A0008DE391E068CE81E891E055CF83E791E02B
:1035B0005DCF6BEC70E08DE391E06CCFCF93DF9348
:1035C0008EE00E94BF0A882309F4B8C08091D80514
:1035D000882309F4B3C0C091A004C111AFC0809189
:1035E000C704811180C080914A04826080934A049C
:1035F0008EE18093350180915F0490E02091620418
:10360000309163048217930728F080914A04806404
:1036100080934A048091D00483FF1DC08091A6044A
:1036200090E005972CF480914A04806280934A04CC
:103630008091A606811105C080914A048061809323
:103640004A048091A506811106C080914A048F7CAE
:10365000886080934A0480914B04811104C080915A
:103660004A0480934B0480914B04282F2195D22F3C
:10367000D8230E94AE2BAB01BC018091AD06909186
:10368000AE06A091AF06B091B0068C509E4FAF4FE2
:10369000BF4F84179507A607B70798F490914B047E
:1036A000992329F08D2F8095892380934B040E94C4
:1036B000AE2B6093AD067093AE068093AF069093E9
:1036C000B00680E090E02D2F30E08830910501F1C8
:1036D000A901082E02C0559547950A94E2F740FDCE
:1036E000C82F0196F2CF80913501882359F090912F
:1036F0009806911123C090914A04946090934A04D3
:10370000815077CF80914A04816080934A0473CFBF
:1037100080914A0490E002978CF0EC2FF0E0EE0FDD
:10372000FF1FEA5CFB4F8591949160918405709135
:1037300085057170DF91CF910C947908DF91CF915D
:1037400008958091A004882381F08250823020F077
:1037500080919706882349F06091840570918505D2
:10376000717082E894E00C946F080895CF93DF9312
:10377000DC01CB01C42FD22F642F70E0625E7D4F3D
:103780004AE00E949032C13051F4E091E505F0E04A
:10379000E15CFE4FED0FF11D808180931E02DF91F1
:1037A000CF910895CF92DF92EF92FF92CF938091C5
:1037B000E105882309F455C085E00E94BF0A8823EB
:1037C00009F44FC08091E505882309F441C0609158
:1037D000B3047091B4048091B5049091B6040E9432
:1037E000273021EA38EF41E550E40E9416310E946B
:1037F000EF2F6B017C01C0910706CC23A9F0C70114
:10380000B6012AE030E040E050E00E943C328C2FCC
:1038100090E0A0E0B0E0281739074A075B0724F0E2
:103820008091970681111DC020E041E0C701B601DB
:103830000E94B61B609172057091730571708EE1E4
:1038400092E0CF91FF90EF90DF90CF900C946F08B3
:10385000C090B304D090B404E090B504F090B604E6
:10386000CACFCF91FF90EF90DF90CF900895CF9285
:10387000DF92EF92FF920F93CF93DF938091BF047B
:10388000882309F471C00E94D21B81E10E94BF0A03
:10389000882309F469C0C090CC04D090CD04E09096
:1038A000CE04F090CF0480911B0690911C0641E05D
:1038B00050E0C114D104E104F10411F040E050E003
:1038C00048235923452B09F04FC04091DF05A0E064
:1038D000B0E08C219D21AE21BF21842B892B8A2B26
:1038E0008B2B09F441C0C0918A05D0918B05D17012
:1038F0008AEC80931E026091BB047091BC0480919D
:10390000BD049091BE0423E5E22E0EE424E04FE1D5
:1039100052E00E949109BE018EE192E00E946F0880
:10392000C0918C05D0918D05D1708BEC80931E02D7
:103930006091B7047091B8048091B9049091BA0471
:1039400037E5E32E05E424E04FE152E00E949109BF
:10395000BE018EE192E0DF91CF910F91FF90EF9049
:10396000DF90CF900C946F08DF91CF910F91FF9073
:10397000EF90DF90CF900895CF93DF938091E5058E
:10398000882309F456C060913E0570913F058091EF
:103990004005909141050E9427302EEA31E646E02D
:1039A0005DE30E9416310E94EF2FEB018091C70466
:1039B000882389F080918E0690918F06069758F0A3
:1039C00080915A0490915B048C179D0724F4D09346
:1039D0005B04C0935A0489E00E94BF0A8823C9F19E
:1039E0008091F8058823A9F12091070630E0211580
:1039F000310561F0CE016AE070E00E940632621784
:103A0000730724F080919706811123C0BE01DD0F5A
:103A1000880B990B20E041E00E94B61B60917A056B
:103A200070917B0571708EE192E0DF91CF910C94E3
:103A30006F0860913E0570913F058091400590911F
:103A4000410524E630E040E050E00E943C32E901CC
:103A5000ADCFDF91CF910895CF92DF92EF92FF9299
:103A6000CF93DF938091BF04882309F460C08091D5
:103A7000E505882309F456C06091C0047091C10423
:103A80008091C2049091C3040E94253021EA38EF4E
:103A900041E550E40E9416310E94F62FEB016E01C1
:103AA000E12CF12C8091560490915704A091580478
:103AB000B09159048C159D05AE05BF0540F4C09228
:103AC0005604D0925704E0925804F092590482E0D0
:103AD0000E94BF0A882359F120910606222369F02B
:103AE000CE0164E670E00E94F23130E062177307A5
:103AF00020F08091970681111AC022E041E0C701B1
:103B0000B6010E94B61B60916C0570916D057170D5
:103B10008EE192E0DF91CF91FF90EF90DF90CF9018
:103B20000C946F08C091C004D091C104B8CFDF914C
:103B3000CF91FF90EF90DF90CF900895E0916601D4
:103B400081E08E0F80936601F0E0E559FE4F8081A1
:103B50000895CF93DF930E949E1DC82FD0E00E944E
:103B60009E1D9E01382BC901DF91CF910895CF9200
:103B7000DF92EF92FF920E94A91D6C01E12CF12CC3
:103B80000E94A91DBC0180E090E0CB017727662749
:103B90006C297D298E299F29FF90EF90DF90CF908F
:103BA000089581E0809331018AE08093330183E0BE
:103BB00080933201109281061092C6048091EB0529
:103BC000882301F110925004109251041092520473
:103BD00010925304109256041092570410925804F5
:103BE0001092590410925B0410925A0410925D04D2
:103BF00010925C04109255041092540410924F04D9
:103C000010924E040C94740326E040E052EC61E004
:103C100070E08AEB96E00E949D2D8091C00082604A
:103C20008093C0001092C50080E18093C4008AEBAD
:103C300096E00E94332D84B18C6284B92498569A00
:103C4000529860E084E10E946B2C60E081E10E9468
:103C50006B2C60E081E10E946B2C61E087E00E94A8
:103C60006B2C0E94DC070E941D050E94E40464EF97
:103C700071E080E090E00E94DF2B8091ED058823C9
:103C800039F081E00E94442B0E9498080C94740340
:103C900083E0F8CFCF93C82F682F8AEB96E00E947D
:103CA000552D809165018C2780936501CF910895F2
:103CB000CF93C92F0E944A1E8C2FCF910C944A1E7D
:103CC000609165018AEB96E00C94552DCF93DF93BC
:103CD000D82FC62F64E28AEB96E00E94552D6DE442
:103CE0008AEB96E00E94552D6CE38AEB96E00E94E9
:103CF000552D109265018C2F0E944A1E8D2F0E9417
:103D00004A1EC11104C0DF91CF910C94601EDF9157
:103D1000CF910895CF92DF92EF92FF920F931F936E
:103D2000CF936EE18AEC0E94661E8EE5C82E85E078
:103D3000D82E94E5E92E95E0F92E0AE415E0C0E0CE
:103D4000F60181916F010E944A1EF70181917F0166
:103D50000E944A1EF80181918F010E944A1ECF5F86
:103D6000CA3071F70E94601E67E08CEC0E94661EEC
:103D7000809149050E944A1E809148050E944A1E72
:103D8000809147050E944A1E809146050E944A1E66
:103D9000809145050E944A1E809144050E944A1E5A
:103DA000809143050E944A1E0E94601E0E94610489
:103DB00060E08AEF0E94661ECF911F910F91FF90E5
:103DC000EF90DF90CF900C94D11D809133018A3019
:103DD000C9F4909132019330A9F4909190069230F9
:103DE0001CF091E090939006909190069F3F1CF4F8
:103DF0009FEF909390069091310120919006920F41
:103E0000909331019091310197FF03C098E0909316
:103E1000310190913101993014F01092310190915B
:103E20003101913071F5EFEFE80FE730A0F4863003
:103E300010F0E1E0E80F209132012230D1F0233080
:103E4000E1F0213041F4F0E0E25AFA4F2081309164
:103E50009006230F20838A3009F03BC290933001F3
:103E600080913201813009F40CC2823009F40BC216
:103E70000895F0E0EC5AFA4FE9CFF0E0E65BFA4F34
:103E8000E5CF923009F042C020913201233019F77A
:103E9000482F50E0FA013197E730F105E0F6EB5A90
:103EA000F04E209190060C945B325C1F621F681FDD
:103EB0006E1F741F7A1F801F30914905230F2093B6
:103EC0004905C9CF30914805230F20934805C3CF3A
:103ED00030914705230F20934705BDCF309146050C
:103EE000230F20934605B7CF30914505230F20932C
:103EF0004505B1CF30914405230F20934405ABCF46
:103F000030914305230F20934305A5CF933009F04B
:103F100050C020913201233009F09DCF482F50E04E
:103F2000FA013197E730F10508F095CFE656F04EEB
:103F30000C945B32A11FA91FB11FB91FC11FC91F5C
:103F4000D11F21E03091CF05311120E02093CF0522
:103F500082CF2091D20530919006230F2093D20575
:103F60007ACF2091D00530919006230F2093D00571
:103F700072CF21E03091D905311120E02093D9058D
:103F80006ACF2091DA0530919006230F2093DA054D
:103F900062CF2091D10530919006230F2093D10557
:103FA0005ACF21E03091D305311120E02093D30581
:103FB00052CF943009F069C120913201233009F0C9
:103FC0004ACF833039F148F48130E1F0823009F092
:103FD00042CF8FE080939B060895853059F110F110
:103FE000863009F038CF209190068091C0059091DD
:103FF000C105820F911D27FD9A959093C10580936D
:10400000C005089581E09091CC05911180E08093E6
:10401000CC05089581E09091CD05911180E08093C9
:10402000CD05089521E03091CE05311120E0209397
:10403000CE0511CF209190068091C2059091C305C5
:10404000820F911D27FD9A959093C3058093C20519
:10405000089520913201233009F0FDCE833051F1D3
:1040600068F48130F9F0823009F0F5CE81E090916A
:10407000D605911180E08093D6050895843011F122
:10408000853009F0E8CE209190068091BC05909192
:10409000BD05820F911D27FD9A959093BD058093D4
:1040A000BC05089581E09091D405911180E0809342
:1040B000D405089581E09091D705911180E0809317
:1040C000D7050895209190068091BE059091BF0577
:1040D000820F911D27FD9A959093BF058093BE0591
:1040E000089520913201233009F0B5CE482F50E0D9
:1040F000FA013197E830F10508F0ADCEEE57FF4DEB
:104100000C945B328A2092209A20A220AA20B2200E
:10411000BA20C22081E09091E805911180E080935F
:10412000E805089581E09091E905911180E0809380
:10413000E905089581E09091F505911180E0809363
:10414000F505089581E09091E705911180E0809355
:10415000E705089581E09091DF05911180E080935B
:10416000DF05089581E09091FC05911180E0809336
:10417000FC05089581E09091F605911180E080930F
:10418000F60508958091EC0590919006890F809333
:10419000EC05089520913201233009F05CCE833084
:1041A00021F168F48130C9F0823009F054CE81E009
:1041B0009091ED05911180E08093ED050895853093
:1041C00001F1D8F0863009F046CE81E09091DB0510
:1041D000911180E08093DB05089581E09091E505E1
:1041E000911180E08093E505089581E09091F405B8
:1041F000911180E08093F40508958AE080939C06F5
:1042000008958091020690919006890F809302068E
:1042100008958091060690919006890F8093060676
:1042200008958091070690919006890F8093070664
:1042300008958091080690919006890F8093080652
:1042400008958091090690919006890F8093090640
:1042500008958091DC0590919006890F8093DC058C
:1042600008958091DD0590919006890F8093DD057A
:10427000089581E09091D805911180E08093D80550
:1042800008950C94D11D0C948A1E953009F4E1CE4A
:10429000963009F426CF973009F47CCF983009F096
:1042A000DACD20913201233009F0D5CD482F50E0EE
:1042B000FA013197E730F10508F0CDCDEE59FE4D0A
:1042C0000C945B320921112119212121292131214D
:1042D000392108950F931F93CF93809112019091EC
:1042E0001301855195408F38914008F062C080914C
:1042F000100190911101855195408F38914008F03F
:1043000058C08091140190911501855195408F38C6
:10431000914008F04EC01092640188EE93E0A0E056
:10432000B0E080935C0190935D01A0935E01B09337
:104330005F0180916401811138C0009112011091D8
:104340001301809181060B3397E0190708F458C0D8
:1043500020911401309115012B33374008F450C0DF
:1043600020911601309117012F37344008F448C0CE
:1043700081111BC080918E0690918F060697A8F040
:104380008091C704811111C082E08093640181E0B3
:104390008093810680913001809331010E947403E3
:1043A00080916401813009F458C0CF911F910F9121
:1043B000089580916401813009F0BBCF0E94AE2B3B
:1043C00000916001109161012091620130916301BF
:1043D000601B710B820B930B00915C0110915D01CE
:1043E00020915E0130915F010617170728073907F2
:1043F00010F4109264018CE291E0A0E0B0E091CF63
:10440000882399F2C0919006109290068091C6047C
:10441000882361F0809116019091170185319540B4
:1044200028F082E0809364010E94D11D8091810672
:10443000882309F454C020911001309111012B33CD
:1044400097E03907C8F081E08093640180913201E0
:104450008F5F843068F4809332010E94AE2B6093AA
:1044600060017093610180936201909363019DCF1D
:1044700083E08093320194CF2E37344050F491E0A2
:104480009093640180913201815029F79093320119
:1044900087CF0B3327E01207A0F091E090936401DF
:1044A00080913301815051F080933301809131012B
:1044B0008111D3CF8AE08093330172CF909333017F
:1044C000F5CF0E37144058F481E080936401809159
:1044D00033018F5F809333018B3060F7BECF9091B3
:1044E000C60491115DCF882309F45ACF8C2FC630B2
:1044F00094F085E020911401309115012E3794E05D
:10450000390768F491E0909364018150809390069C
:104510000E94E51E45CFCB3F6CF78BEFEBCF2B33E3
:10452000374008F43DCF91E0909364018F5F809312
:10453000900680913101883059F7809132018330A3
:1045400039F780913301853019F710929C06E0CF3E
:104550000F931F93CF936FE18CED0E94661E89E04D
:104560000E944A1EC0E00091450610914606C8010F
:104570000E94C53280934406C8010E94581E809153
:1045800044060E944A1E8091450690914606019677
:104590009093460680934506CF5FCA3021F7CF91AE
:1045A0001F910F910C94601E63E08CED0E94661EBB
:1045B00089E00E944A1E80914506909146060E941D
:1045C000581E0C94601ECF92DF92EF92FF920F93D1
:1045D0001F93CF93DF938091A9069091AA0601962D
:1045E0009093AA068093A9061092660183E08093B7
:1045F000A506809168018C3D79F50E949E1D893049
:1046000009F099C00E949E1D90E090934606809309
:1046100045060E949E1D2091450630914606280FB2
:10462000311D30934606209345060E949E1D8093BF
:10463000440681E0809343060E94AE2B6854744F79
:104640008F4F9F4F60933F067093400680934106C3
:10465000909342060E94A82280916801843609F056
:104660003DC181E0809391060E949E1D8093CB0402
:10467000809168018A3609F07AC185E08093A606A8
:104680000E949E1D882319F081E08093BF040E9440
:104690009E1D8093A6040E94B71D6093BB04709377
:1046A000BC048093BD049093BE040E94B71D609328
:1046B000B7047093B8048093B9049093BA040E942D
:1046C000A91DA0E0B0E02091C70421110BC0809388
:1046D000AF049093B004A093B104B093B20421E06E
:1046E000209384064091AF045091B0046091B104CE
:1046F0007091B204841B950BA60BB70B8093B30487
:104700009093B404A093B504B093B6040E94A91D7D
:104710009093AE048093AD040E94A91D9093AC04C5
:104720008093AB04DF91CF911F910F91FF90EF9099
:10473000DF90CF900895883009F055C0C0E0D1E0F7
:104740000E949E1D90E090934606809345060E942D
:104750009E1D90E0982F88272091450630914606AF
:10476000820F931F90934606809345060E949E1DDC
:1047700080934406D09343060E94AE2B6854744F36
:104780008F4F9F4F60933F06709340068093410682
:1047900090934206609144068091450690914606AA
:1047A0000E943C036CE080E090E00E943C0380911A
:1047B0004506909146068935910519F08F34914050
:1047C00011F40E94E404CF5FCA3009F0B9CF8091A0
:1047D00045069091460601969093460680934506BD
:1047E0000E94D42239CF8730E1F56BE08CED0E9436
:1047F000661E87E00E944A1EC2EED4E085E0C63401
:10480000D80759F08881998143E0969587954A9514
:10481000E1F70E94581E6496F1CF0E94601E6DE081
:104820008CED0E94661E8AE00E944A1E84E090E0A1
:104830000E94581E82E090E00E94581E80E996E097
:104840000E94581E80E090E00E94581E80E090E098
:104850000E94581E81E090E00E94581E0E94601E37
:10486000FBCE833071F580916901853089F40E9417
:10487000A91D80329D4109F0EFCE0E949E1D8093BC
:1048800049060E949E1D809348060E946103E4CE63
:10489000883309F0E1CE0AE416E0C0E00E949E1DD4
:1048A000F80181938F01CF5FC633C1F70E949E1D2F
:1048B000C82F0E94F208CF3F09F0CECE0E94980880
:1048C000CBCE863041F40E9459080E941D0581E03C
:1048D00080939306C1CE8530D1F3BECE8536A9F53F
:1048E0000E94A91D90938D0680938C060E94A91D9D
:1048F00090938B0680938A060E94A91D9093D10401
:104900008093D0040E94B71D6093CC047093CD04B3
:104910008093CE049093CF0420911406022F10E0D0
:1049200020E030E0DC01CB0180239123A223B323DC
:1049300021E0892B8A2B8B2B09F420E02093C704DC
:104940000E949E1D8093420593CE893609F090CE39
:1049500000E111E0C1E00E94A91DD8018D939D9353
:104960008D01CF5FC930B9F70E946A2181CE8B36A5
:1049700099F40E94A91DA0E0B0E08093C004909338
:10498000C104A093C204B093C3040E94A91D9093D4
:10499000A8048093A704C6CE893759F40E949E1DAF
:1049A0000E949E1D0E949E1D0E949E1D8093A50434
:1049B000B9CE8C36C1F40E94A91D9093370580931F
:1049C00036050E94A91D90933905809338050E94F1
:1049D000A91D843B910514F088569140909373046F
:1049E000809372049FCE8D3689F40E94B71D609328
:1049F0003E0570933F0580934005909341050E94CA
:104A0000A91D9093C9048093C8048CCE8E3609F0FA
:104A1000B5C10E949E1D8093CA040E94A91D909357
:104A2000A4048093A3040E94A91D9093A2048093E0
:104A3000A1040E94A91D909369048093680472CE1A
:104A40008537D1F5F12C02E114E0C7E0D0E02F2D3D
:104A500030E08091690190E0281739071CF50E9429
:104A60009E1D9BEF9D0F9230D0F02D2F30E029300E
:104A70003105ACF48B3351F4F80110828C2F90E0A7
:104A80000196080F191FC7E0DF5F07C0CC2329F08C
:104A9000D8018C93C1500F5F1F4FF394D8CF8B3345
:104AA000E1F7F2CF80911A0290911B02A0911C02B3
:104AB000B0911D02AF7D8AC1803739F52EE5C22E37
:104AC00025E0D22E34E5E32E35E0F32E0AE415E09E
:104AD000C0E00E949E1DF60181936F010E949E1D01
:104AE000D7018D937D010E949E1DF80181938F0156
:104AF000CF5FCA3071F780911A0290911B02A0918A
:104B00001C02B0911D029B7F61C1823F41F50E9452
:104B10009E1D8093A0048091690190E0EC01219793
:104B20004E97D4F4CE018E579B4FDC011C9210E0BF
:104B3000E12EF12CEC16FD060CF0F4CD0E949E1D2A
:104B400097012E31310514F02DE130E02E573B4F07
:104B5000F90180831F5FECCF8DE190E0E4CF8737D0
:104B600009F0E0CD81E0809392061091690185E221
:104B7000E4E1F6E0DF011D928A95E9F7C12CD12C22
:104B80007601C394CDE1D0E0112309F4CBCD0E948E
:104B90009E1D90E0C817D90708F428C0FC01ED520B
:104BA000FA4D0C945B32F125FC2502260826F625E9
:104BB0000E26F625F6251426F6251F262A26352646
:104BC000F625F625F6254026F625F62555266A26ED
:104BD0007F26F625F625F625F625F625F6259426D4
:104BE000A926809114068C2980931406CC0CDD1C18
:104BF000EE1CFF1C1150C8CF809115068C298093A4
:104C00001506F4CF809116068C2980931606EECFF8
:104C1000809117068C2980931706E8CF809118069B
:104C20008C2980931806E2CF8091190690911A067C
:104C30008C299D2990931A0680931906D7CF8091CD
:104C40001B0690911C068C299D2990931C0680932D
:104C50001B06CCCF80911D0690911E068C299D29A4
:104C600090931E0680931D06C1CF80911F069091E0
:104C700020068C299D299093200680931F06B6CF8D
:104C800080912D0690912E06A0912F06B0913006AE
:104C90008C299D29AE29BF2980932D0690932E063D
:104CA000A0932F06B0933006A1CF80912906909152
:104CB0002A06A0912B06B0912C068C299D29AE299D
:104CC000BF298093290690932A06A0932B06B093C0
:104CD0002C068CCF8091310690913206A09133063C
:104CE000B09134068C299D29AE29BF2980933106C5
:104CF00090933206A0933306B093340677CF809119
:104D0000350690913606A0913706B09138068C2969
:104D10009D29AE29BF298093350690933606A0932E
:104D20003706B093380662CF809121069091220613
:104D3000A0912306B09124068C299D29AE29BF2974
:104D40008093210690932206A0932306B093240615
:104D50004DCF8091250690912606A0912706B0910F
:104D600028068C299D29AE29BF298093250690937A
:104D70002606A0932706B093280638CF8F3609F071
:104D80005FCE0E949E1D809349050E949E1D8093C8
:104D900048050E949E1D809347050E949E1D80939A
:104DA00046050E949E1D809345050E949E1D80938E
:104DB00044050E949E1D8093430580911A029091A4
:104DC0001B02A0911C02B0911D029D7F80931A02CC
:104DD00090931B02A0931C02B0931D02A3CCFF92E0
:104DE0000F931F93CF93DF93F82E8AEB96E00E94E8
:104DF000D62C892B31F4DF91CF911F910F91FF9029
:104E00000895C5E0D0E004E010E013C02130310582
:104E100069F58D3441F582E090E090935B018093D9
:104E20005A018AEB96E00E94D62C892B21F3FF20B1
:104E300011F38AEB96E00E94F02C482F2091AB06EC
:104E40003091AC062F5F3F4F3093AC062093AB06FA
:104E500020915A0130915B0121153105B9F681E0AD
:104E600090E04432D1F280E090E0D7CF223031059B
:104E700029F48E33C1F783E090E0CFCF23303105A2
:104E800099F49C013327273931052CF010925B01EE
:104E900010925A01C6CF8093690110935B01009371
:104EA0005A0180936701BDCF2430310571F4D0934E
:104EB0005B01C0935A018093680190916701892733
:104EC0008093670110926A01ACCF2530310509F05B
:104ED000A8CF20916701322F382730936701E091E6
:104EE0006A0130916901E31305C08213CFCF0E949C
:104EF000E322CCCF91E09E0F90936A01F0E0E55958
:104F0000FE4F80838ECFCF92DF92EF92FF920E946E
:104F1000AE2B6B017C0128E2C20ED11CE11CF11CFE
:104F200081E08093010280910102882371F00E9448
:104F3000AE2BC616D706E806F90618F41092010241
:104F4000F2CF80E00E94EF26EECFFF90EF90DF904F
:104F5000CF900895FF920F931F93CF93DF935E98A6
:104F600060E085E00E94900860E086E00E94900882
:104F700061E084E00E9490080E94832702E312E02F
:104F8000C0E0D0E080E2F82E80910302909104020C
:104F9000C817D90778F4C03FD10511F40E948327C0
:104FA000F801608187E00E949008F801F1928F017A
:104FB0002196EACF6FEF87E00E94900860E084E0DE
:104FC0000E9490085E9ADF91CF911F910F91FF9000
:104FD0000895CF92DF92EF92FF9210924A0480914F
:104FE000A7069091A80601969093A8068093A7061D
:104FF00080919306882311F00C940000E091020642
:10500000E09334011092830680910106882309F40D
:10501000CCC1F0E0EE0FFF1FE25FFE4F8081918177
:10502000813426E0920708F4BAC181E080938306B8
:10503000909183068091820698130E949604809135
:105040008306809382068091950690E006970CF483
:10505000C6C161E087E00E94A72C0E94AE2B6B01C5
:105060007C018091120290911302A0911402B091E0
:105070001502B701A601481B590B6A0B7B0B44367E
:1050800051056105710508F445C08C599F4FAF4F1C
:10509000BF4F8093120290931302A0931402B09317
:1050A0001502809195068F5F8093950680919606F4
:1050B0008F5F8093960681E090919806911180E031
:1050C000809398060E9416048091D6058823D1F01B
:1050D00020916E0430916F044091700450917104DE
:1050E00060916A0470916B0480916C0490916D04DE
:1050F0000E94072F60936A0470936B0480936C0482
:1051000090936D0480918006811104C060E08CE66C
:105110000E94661E80910E0290910F02A0911002D3
:10512000B0911102C81AD90AEA0AFB0A22E3C21690
:10513000D104E104F10408F48CC0C296A11DB11D94
:1051400080930E0290930F02A0931002B09311026D
:105150008091160290911702A0911802B091190245
:10516000892B8A2B8B2B81F480911A0290911B0240
:10517000A0911C02B0911D02809316029093170219
:10518000A0931802B0931902C0901602D090170293
:10519000E0901802F090190288279927DC018C19F9
:1051A0009D09AE09BF098C219D21AE21BF21AC0113
:1051B000BD0140955095609570954C215D216E2103
:1051C0007F21409316025093170260931802709348
:1051D0001902811522E09207A105B10509F448C121
:1051E00008F011C180319105A105B10509F43AC15A
:1051F00008F0F7C082309105A105B10509F42CC172
:1052000088309105A105B10509F428C10197A105D0
:10521000B10509F037C184E690918006911105C06F
:1052200060E00E94661E0E94AA270E948D05809160
:105230008E0690918F06059708F026C10E944A12AB
:105240008091760490917704CC9790939A068093FE
:1052500099068091960690E005974CF0109296067C
:1052600081E090919706911180E0809397060E94CB
:10527000AE2BAB01BC018091A1069091A206A0913A
:10528000A306B091A40688519C4FAF4FBF4F84171F
:105290009507A607B70708F07BC08093A1069093F7
:1052A000A206A093A306B093A4061092950680913F
:1052B000A7069091A80690933E0680933D06109213
:1052C000A8061092A7068091A9069091AA0690932D
:1052D0003C0680933B061092AA061092A906809184
:1052E000AB069091AC0690933A06809339061092E3
:1052F000AC061092AB0680917604909177040196EB
:10530000909377048093760480918006811102C087
:105310000E942F098091A606811198C11092A604BF
:105320008091A506882319F081508093A50680916D
:10533000C70481118FC1809172049091730490937E
:10534000C5048093C40480918E0690918F060196C7
:1053500090938F0680938E0680919C06813051F445
:1053600080918106882331F060E08EEC0E94661EF9
:1053700010929C0680919C06882319F0815080939E
:105380009C0680919B06882319F0815080939B0690
:1053900081E0FF90EF90DF90CF900C94EF2689375B
:1053A000954008F445CE82E041CE80912906909147
:1053B0002A06A0912B06B0912C064091CC04509166
:1053C000CD046091CE047091CF0484239523A6234D
:1053D000B723892B8A2B8B2B09F027CE29CE60E0AF
:1053E00039CE80389105A105B105D1F1811521E0B3
:1053F0009207A105B105C1F18097A105B10509F09A
:1054000041C08BE609CF009721E0A207B10571F1F9
:1054100098F4811528E09207A105B10579F181156D
:1054200020E19207A105B10559F181159440A1052C
:10543000B10541F580E7F0CE009724E0A207B10561
:10544000C9F0009720E2A207B105B1F00097A24091
:10545000B105C1F482EFE0CE85E6DECE89E6DCCE92
:105460008AE6DACE8DE6D8CE8EE6D6CE82E7D4CEE8
:105470008FE6D2CE8BE3D0CE85E7CECE87E7CCCEFB
:105480008CEDCACE80E0C8CE8091C704882349F055
:1054900081E08093C60480918106813031F40E94BE
:1054A000D11D8091C604882381F08091C7048111A9
:1054B0000CC0109231018AE08093330181E0809327
:1054C0003201809381060E947403809181068823B3
:1054D00019F00E94F016BDCE0E9474038091D00492
:1054E00080FF0AC0609138057091390580913605BA
:1054F000909137050E94CD0C8091CF0581110E94BB
:10550000530F8091D90581110E94E30F8091CC0542
:10551000882379F08091CB0590E02091660430914A
:105520006704821793071CF08091970681110E94EF
:10553000C4118091D405882321F120E030E040E2BD
:1055400051E460916E0470916F04809170049091A9
:1055500071040E947D2F6B017C016091DD0570E07C
:1055600080E090E00E9427309B01AC01C701B601AA
:105570000E94732F87FD03C08091970681110E94BE
:1055800011118091D605882349F00E943E0388239B
:1055900009F477C080919706811173C00E94BD10F5
:1055A0000E945B110E94DE1A8091E70581110E9422
:1055B00017108091990690919A0620917604309167
:1055C0007704AC01445C5F4F42175307A0F4805C42
:1055D0009F4F8217930720F430939A0620939906E1
:1055E0008091F005882339F08091B6059091B70538
:1055F00091700E94BC0C8091D00482FF04C00E9474
:1056000025120E94EF118091D00481FF04C00E94F6
:10561000BC1C0E941E138091D00483FF12C0809195
:10562000DE05882371F00E9483120E94AA130E9453
:105630002C1D0E9484130E94AE120E94371C0E94EF
:10564000B7140E94CF0A0E94A11B03CE8150809301
:10565000A60666CE8091740490917504019690938D
:1056600075048093740480914E0490914F040196C8
:1056700090934F0480934E04109281060E9474030D
:1056800062CE0E949B118ACF8093360108958E309E
:1056900008F08E502091360190E4299F900111244A
:1056A0008770822B80937C0080917A008064809345
:1056B0007A0080917A0086FDFCCF8091780020915D
:1056C000790090E0922B08951F920F920FB60F92DF
:1056D00011242F933F938F939F93AF93BF93809108
:1056E000B2069091B306A091B406B091B506309180
:1056F000B10623E0230F2D3758F50196A11DB11DEA
:105700002093B1068093B2069093B306A093B4069B
:10571000B093B5068091B6069091B706A091B806F1
:10572000B091B9060196A11DB11D8093B606909364
:10573000B706A093B806B093B906BF91AF919F91F9
:105740008F913F912F910F900FBE0F901F90189542
:1057500026E8230F0296A11DB11DD2CF2FB7F894D2
:105760006091B2067091B3068091B4069091B5062F
:105770002FBF08953FB7F8948091B6069091B70671
:10578000A091B806B091B90626B5A89B05C02F3FD9
:1057900019F00196A11DB11D3FBFBA2FA92F982F57
:1057A0008827BC01CD01620F711D811D911D42E052
:1057B000660F771F881F991F4A95D1F70895CF92DA
:1057C000DF92EF92FF92CF93DF936B017C010E94F7
:1057D000BA2BEB01C114D104E104F10439F4DF91D7
:1057E000CF91FF90EF90DF90CF9008950E94D52C3D
:1057F0000E94BA2B6C1B7D0B683E734058F381E00E
:10580000C81AD108E108F108C851DC4FE3CF7894F9
:1058100084B5826084BD84B5816084BD85B58260B5
:1058200085BD85B5816085BDEEE6F0E08081816053
:105830008083E1E8F0E01082808182608083808153
:1058400081608083E0E8F0E0808181608083E1EB2B
:10585000F0E0808184608083E0EBF0E08081816013
:105860008083EAE7F0E080818460808380818260C9
:1058700080838081816080838081806880831092B2
:10588000C1000895833081F028F4813099F082308E
:10589000A9F008958730A9F08830C9F08430B1F4B8
:1058A000809180008F7D03C0809180008F778093EE
:1058B0008000089584B58F7784BD089584B58F7D69
:1058C000FBCF8091B0008F778093B00008958091D6
:1058D000B0008F7DF9CFCF93DF9390E0FC01EF52C2
:1058E000FA4F24918B519A4FFC0184918823C9F07F
:1058F00090E0880F991FFC01ED5FF94FA591B491DD
:10590000FC01E750FA4FC591D49161110DC09FB7CA
:10591000F8948C91209582238C9388812823288366
:105920009FBFDF91CF910895623051F49FB7F894F3
:105930003C91822F809583238C93E8812E2BEFCF8F
:105940008FB7F894EC912E2B2C938FBFEACF1F9337
:10595000CF93DF93162F282F30E0F901E354FA4F4D
:105960008491F901EF52FA4FD491F901EB51FA4FBA
:10597000C491CC23A1F081110E94422CEC2FF0E0C5
:10598000EE0FFF1FE750FA4FA591B4918FB7F8942F
:10599000EC91111108C0D095DE23DC938FBFDF910D
:1059A000CF911F910895DE2BF8CF0895FC01918DC2
:1059B000228D892F90E0805C9F4F821B91098F730D
:1059C00099270895FC01918D828D981731F0828D71
:1059D000E80FF11D858D90E008958FEF9FEF0895FA
:1059E000FC01918D828D981761F0828DDF01A80FE7
:1059F000B11D5D968C91928D9F5F9F73928F90E009
:105A000008958FEF9FEF089586E59EE2892B49F078
:105A100080E090E0892B29F00E94562E81110C9491
:105A200000000895FC01848DDF01A80FB11DA35A69
:105A3000BF4F2C91848D90E001968F739927848FAE
:105A4000A689B7892C93A089B1898C9180648C93A5
:105A5000938D848D981306C00288F389E02D808190
:105A60008F7D80830895CF93DF93EC01888D882309
:105A700051F0EA89FB89808185FD08C0A889B98930
:105A80008C9186FF03C0DF91CF9108950FB607FC7C
:105A9000F2CF808185FFEFCFA889B9898C9185FFEE
:105AA000EACFCE010E94122DE4CFEF92FF920F9326
:105AB0001F93CF93DF93EC01F62E9B8D8C8D981363
:105AC00005C0E889F989808185FD2EC00B8D10E025
:105AD0000F5F1F4F0F731127E02E8C8DE8120CC043
:105AE0000FB607FCFACFE889F989808185FFF5CFE9
:105AF000CE010E94122DF1CF8B8DFE01E80FF11D1A
:105B0000E35AFF4FF0820B8FEA89FB898081806224
:105B1000808381E0888F81E090E0DF91CF911F91B9
:105B20000F91FF90EF900895EE89FF896083E889D7
:105B3000F989808180648083EECFCF92DF92EF92EB
:105B4000FF921F93CF93DF93EC016A017B01122F29
:105B5000E889F98982E080834115514E610571051C
:105B6000A1F060E079E08DE390E0A70196010E944A
:105B70001A322150310941095109569547953795F7
:105B80002795211580E1380798F0E889F989108276
:105B900060E874E88EE190E0A70196010E941A3255
:105BA0002150310941095109569547953795279557
:105BB000EC85FD853083EE85FF852083188EEC898A
:105BC000FD891083EA89FB89808180618083EA896D
:105BD000FB89808188608083EA89FB898081806875
:105BE0008083EA89FB8980818F7D8083DF91CF91DB
:105BF0001F91FF90EF90DF90CF9008951F920F922A
:105C00000FB60F9211242F938F939F93EF93FF93CF
:105C1000E091CA06F091CB068081E091D006F09128
:105C2000D10682FD1BC090818091D3068F5F8F7358
:105C30002091D406821741F0E091D306F0E0E654BB
:105C4000F94F958F8093D306FF91EF919F918F919C
:105C50002F910F900FBE0F901F9018958081F4CF59
:105C60001F920F920FB60F9211242F933F934F93D1
:105C70005F936F937F938F939F93AF93BF93EF93B4
:105C8000FF938AEB96E00E94122DFF91EF91BF9156
:105C9000AF919F918F917F916F915F914F913F91C4
:105CA0002F910F900FBE0F901F9018958AEB96E0E2
:105CB0000E94D62C21E0892B09F420E0822F089540
:105CC000EAEBF6E01382128288EE93E0A0E0B0E007
:105CD00084839583A683B7838DE491E09183808349
:105CE00085EC90E09587848784EC90E097878687A1
:105CF00080EC90E0918B808B81EC90E0938B828B99
:105D000082EC90E0958B848B86EC90E0978B868B71
:105D1000118E128E138E148E08954F925F926F9291
:105D20007F92AF92BF92CF92DF92EF92FF920F934A
:105D30001F93CF93DF93CDB7DEB729013A019B01C3
:105D4000AC01241935094609570989899A89AB8913
:105D5000BC89BC01CD016A197B098C099D090E948F
:105D6000D431A801970124193509460957090E9421
:105D70003C32CA01B9016A0D7B1D8C1D9D1DDF914E
:105D8000CF911F910F91FF90EF90DF90CF90BF9038
:105D9000AF907F906F905F904F90089508950E940C
:105DA000072C0E94CE2E0E94041EC4E0DDE20E9459
:105DB000E9272097E1F30E94042DF9CFCF92DF92DB
:105DC000EF92FF920F931F93CF93DF936C01EB0140
:105DD0007B01E40EF51E00E010E0CE15DF0561F05A
:105DE0006991D601ED91FC910190F081E02DC60101
:105DF0000995080F191FF1CFC801DF91CF911F91AD
:105E00000F91FF90EF90DF90CF9008955058BB27EF
:105E1000AA270E941E2F0C94C8300E948F3038F0A1
:105E20000E94963020F039F49F3F19F426F40C9428
:105E30008C300EF4E095E7FB0C948630E92F0E943D
:105E4000ED3058F3BA17620773078407950720F0FF
:105E500079F4A6F50C940F310EF4E0950B2EBA2FC1
:105E6000A02D0B01B90190010C01CA01A001112460
:105E7000FF27591B99F0593F50F4503E68F11A160C
:105E8000F040A22F232F342F4427585FF3CF46959D
:105E900037952795A795F0405395C9F77EF41F16BF
:105EA000BA0B620B730B840BBAF09150A1F0FF0F89
:105EB000BB1F661F771F881FC2F70EC0BA0F621F75
:105EC000731F841F48F4879577956795B795F79565
:105ED0009E3F08F0B0CF9395880F08F09927EE0FFA
:105EE0009795879508950E94623008F481E008959F
:105EF0000E949F30E3950C94D9300E94912F0C940E
:105F0000C8300E94963058F00E948F3040F029F43B
:105F10005F3F29F00C94863051110C9410310C9491
:105F20008C300E94ED3068F39923B1F3552391F33F
:105F3000951B550BBB27AA2762177307840738F0F8
:105F40009F5F5F4F220F331F441FAA1FA9F335D055
:105F50000E2E3AF0E0E832D091505040E695001C09
:105F6000CAF72BD0FE2F29D0660F771F881FBB1FC3
:105F7000261737074807AB07B0E809F0BB0B802DA1
:105F8000BF01FF2793585F4F3AF09E3F510578F0CD
:105F90000C9486300C9410315F3FE4F3983ED4F3B8
:105FA000869577956795B795F7959F5FC9F7880FA1
:105FB000911D9695879597F90895E1E0660F771FF3
:105FC000881FBB1F621773078407BA0720F0621B84
:105FD000730B840BBA0BEE1F88F7E09508950E94AF
:105FE000F62F6894B1110C94103108950E94F53089
:105FF00088F09F5798F0B92F9927B751B0F0E1F08A
:10600000660F771F881F991F1AF0BA95C9F714C039
:10601000B13091F00E940F31B1E008950C940F312E
:10602000672F782F8827B85F39F0B93FCCF3869572
:1060300077956795B395D9F73EF4909580957095CF
:1060400061957F4F8F4F9F4F0895E89409C097FB4C
:106050003EF490958095709561957F4F8F4F9F4F3F
:106060009923A9F0F92F96E9BB279395F695879583
:1060700077956795B795F111F8CFFAF4BB0F11F446
:1060800060FF1BC06F5F7F4F8F4F9F4F16C08823ED
:1060900011F096E911C0772321F09EE8872F762F23
:1060A00005C0662371F096E8862F70E060E02AF064
:1060B0009A95660F771F881FDAF7880F9695879550
:1060C00097F90895990F0008550FAA0BE0E8FEEF25
:1060D00016161706E807F907C0F012161306E407AC
:1060E000F50798F0621B730B840B950B39F40A26A5
:1060F00061F0232B242B252B21F408950A2609F483
:10610000A140A6958FEF811D811D089597F99F6786
:1061100080E870E060E008959FEF80EC089500242F
:106120000A941616170618060906089500240A94FC
:10613000121613061406050608950C948C300E945E
:10614000F530D8F3E894E0E0BB279F57F0F02AED54
:106150003FE049EC06C0EE0FBB0F661F771F881F9C
:1061600028F0B23A62077307840728F0B25A620B2C
:10617000730B840BE3959A9572F7803830F49A95F7
:10618000BB0F661F771F881FD2F790480C948D3184
:10619000092E0394000C11F4882352F0BB0F40F435
:1061A000BF2B11F460FF04C06F5F7F4F8F4F9F4F75
:1061B0000895EF93E0FF07C0A2EA2AED3FE049EC23
:1061C0005FEB0E941E2F0E94C8300F90039401FCC9
:1061D0009058E8E6F0E00C94993157FD9058440F40
:1061E000551F59F05F3F71F04795880F97FB991F36
:1061F00061F09F3F79F087950895121613061406F3
:10620000551FF2CF4695F1DF08C01616170618067F
:10621000991FF1CF86957105610508940895E8945A
:10622000BB2766277727CB0197F908950E9429316C
:106230000C94C8300E948F3038F00E94963020F0C5
:10624000952311F00C9486300C948C3011240C940E
:1062500010310E94ED3070F3959FC1F3950F50E01F
:10626000551F629FF001729FBB27F00DB11D639F08
:10627000AA27F00DB11DAA1F649F6627B00DA11DAE
:10628000661F829F2227B00DA11D621F739FB00D54
:10629000A11D621F839FA00D611D221F749F3327C4
:1062A000A00D611D231F849F600D211D822F762F5D
:1062B0006A2F11249F5750409AF0F1F088234AF03A
:1062C000EE0FFF1FBB1F661F771F881F91505040A6
:1062D000A9F79E3F510580F00C9486300C94103144
:1062E0005F3FE4F3983ED4F3869577956795B7952D
:1062F000F795E7959F5FC1F7FE2B880F911D969547
:10630000879597F908959F930E949F300F9007FCFF
:10631000EE5F0C94D9309F3F31F0915020F4879577
:1063200077956795B795880F911D9695879597F9FD
:1063300008959F938F937F936F93FF93EF939B01A8
:10634000AC010E941631EF91FF910E94AD312F9167
:106350003F914F915F910C941631DF93CF931F9330
:106360000F93FF92EF92DF927B018C01689406C03D
:10637000DA2EEF010E942931FE01E894A5912591C2
:10638000359145915591A6F3EF010E941E2FFE0114
:106390009701A801DA9469F7DF90EF90FF900F91D1
:1063A0001F91CF91DF910895DB018F939F930E94FE
:1063B0006132BF91AF91A29F800D911DA39F900D5F
:1063C000B29F900D1124089587FB082E062687FDA5
:1063D000819567FD61950E946C320EF4919507FCE2
:1063E00081950895AA1BBB1B51E107C0AA1FBB1FC3
:1063F000A617B70710F0A61BB70B881F991F5A9551
:10640000A9F780959095BC01CD01089597FB072EC3
:1064100016F4009407D077FD09D00E94F23107FCF2
:1064200005D03EF4909581959F4F089570956195A4
:106430007F4F0895A1E21A2EAA1BBB1BFD010DC0C0
:10644000AA1FBB1FEE1FFF1FA217B307E407F50724
:1064500020F0A21BB30BE40BF50B661F771F881F00
:10646000991F1A9469F760957095809590959B0196
:10647000AC01BD01CF010895052E97FB1EF40094D9
:106480000E94533257FD07D00E941A3207FC03D0F6
:106490004EF40C94533250954095309521953F4FD2
:1064A0004F4F5F4F089590958095709561957F4F00
:1064B0008F4F9F4F0895EE0FFF1F0590F491E02D31
:1064C00009940E947832A59F900DB49F900DA49FCF
:1064D000800D911D11240895991B79E004C0991F26
:1064E000961708F0961B881F7A95C9F7809508952E
:1064F000A29FB001B39FC001A39F700D811D112405
:10650000911DB29F700D811D1124911D0895FB01F5
:10651000DC0102C005900D9241505040D8F708951B
:10652000BB274A3031F4992322F4BDE2909581953E
:106530009F4F0C949C32BB27FB015527AA27880F3D
:10654000991FAA1FA41710F0A41B83955051B9F7E7
:10655000A05DAA3308F0A95DA193009779F7B11166
:10656000B1931192CB010C94B532DC01FC01672F81
:1065700071917723E1F7329704C07C916D9370831A
:106580006291AE17BF07C8F30895F999FECF92BD87
:1065900081BDF89A992780B50895262FF999FECFE5
:1065A0001FBA92BD81BD20BD0FB6F894FA9AF99A30
:0A65B0000FBE01960895F894FFCF86
:1065BA00010E100F11116C074C0410102A22DC0571
:1065CA00DC05DC05DC05DC05DC05DC05DC05DC05B9
:1065DA00DC05DC05DC05DC05DC05DC05DC0500008A
:1065EA000101030A081E015000490044002D00A7BA
:1065FA00A8BBB97AA7DFBBA5A600000000552DDE0F
:0A660A002ED62CF02CE22C332D00CC
:00000001FF
